 setenvstor001

 Timestamp is 467c108a (reproducible build file hash)

 Preferred load address is 0000000180000000

 Start         Length     Name                   Class
 0001:00000000 00003750H .text$mn                CODE
 0001:00003750 00000036H .text$mn$00             CODE
 0001:00003786 00000092H .text$x                 CODE
 0002:00000000 000001c8H .idata$5                DATA
 0002:000001c8 00000038H .00cfg                  DATA
 0002:00000200 00000008H .CRT$XCA                DATA
 0002:00000208 00000008H .CRT$XCZ                DATA
 0002:00000210 00000008H .CRT$XIA                DATA
 0002:00000218 00000008H .CRT$XIC                DATA
 0002:00000220 00000008H .CRT$XIZ                DATA
 0002:00000228 00000008H .CRT$XLA                DATA
 0002:00000230 00000008H .CRT$XLZ                DATA
 0002:00000238 00000008H .CRT$XPA                DATA
 0002:00000240 00000008H .CRT$XPZ                DATA
 0002:00000248 00000008H .CRT$XTA                DATA
 0002:00000250 00000010H .CRT$XTZ                DATA
 0002:00000258 00000000H .gehcont$y              DATA
 0002:00000258 00000000H .gfids$y                DATA
 0002:00000260 000022a0H .rdata                  DATA
 0002:00002500 00000000H .rdata$CastGuardVftablesA DATA
 0002:00002500 00000000H .rdata$CastGuardVftablesC DATA
 0002:00002500 00000028H .rdata$T                DATA
 0002:00002528 000000e8H .rdata$voltmd           DATA
 0002:00002610 00000320H .rdata$zzzdbg           DATA
 0002:00002930 00000008H .rtc$IAA                DATA
 0002:00002938 00000008H .rtc$IZZ                DATA
 0002:00002940 00000008H .rtc$TAA                DATA
 0002:00002948 00000008H .rtc$TZZ                DATA
 0002:00002950 00000004H .tls                    DATA
 0002:00002954 00000004H .tls$                   DATA
 0002:00002958 00000008H .tls$ZZZ                DATA
 0002:00002960 00000370H .xdata                  DATA
 0002:00002cd0 00000398H .edata                  DATA
 0002:00003068 0000008cH .idata$2                DATA
 0002:000030f4 00000014H .idata$3                DATA
 0002:00003108 000001c8H .idata$4                DATA
 0002:000032d0 00000486H .idata$6                DATA
 0003:00000000 00000090H .data                   DATA
 0003:00000090 0001b638H .bss                    DATA
 0004:00000000 000003f0H .pdata                  DATA

  Address         Publics by Value              Rva+Base               Lib:Object

 0000:00000000       __AbsoluteZero             0000000000000000     <absolute>
 0000:00000000       ___safe_se_handler_count   0000000000000000     <absolute>
 0000:00000000       ___safe_se_handler_table   0000000000000000     <absolute>
 0000:00000000       __arm64x_extra_rfe_table   0000000000000000     <absolute>
 0000:00000000       __arm64x_extra_rfe_table_size 0000000000000000     <absolute>
 0000:00000000       __arm64x_native_entrypoint 0000000000000000     <absolute>
 0000:00000000       __arm64x_redirection_metadata 0000000000000000     <absolute>
 0000:00000000       __arm64x_redirection_metadata_count 0000000000000000     <absolute>
 0000:00000000       __dynamic_value_reloc_table 0000000000000000     <absolute>
 0000:00000000       __enclave_config           0000000000000000     <absolute>
 0000:00000000       __guard_check_icall_a64n_fptr 0000000000000000     <absolute>
 0000:00000000       __guard_eh_cont_count      0000000000000000     <absolute>
 0000:00000000       __guard_eh_cont_table      0000000000000000     <absolute>
 0000:00000000       __guard_fids_count         0000000000000000     <absolute>
 0000:00000000       __guard_fids_table         0000000000000000     <absolute>
 0000:00000000       __guard_iat_count          0000000000000000     <absolute>
 0000:00000000       __guard_iat_table          0000000000000000     <absolute>
 0000:00000000       __guard_longjmp_count      0000000000000000     <absolute>
 0000:00000000       __guard_longjmp_table      0000000000000000     <absolute>
 0000:00000000       __hybrid_auxiliary_iat     0000000000000000     <absolute>
 0000:00000000       __hybrid_auxiliary_iat_copy 0000000000000000     <absolute>
 0000:00000000       __hybrid_code_map          0000000000000000     <absolute>
 0000:00000000       __hybrid_code_map_count    0000000000000000     <absolute>
 0000:00000000       __x64_code_ranges_to_entry_points 0000000000000000     <absolute>
 0000:00000000       __x64_code_ranges_to_entry_points_count 0000000000000000     <absolute>
 0000:00000100       __guard_flags              0000000000000100     <absolute>
 0000:00000000       __ImageBase                0000000180000000     <linker-defined>
 0001:00000000       ?NewObject@JNIEnv_@@QEAAPEAV_jobject@@PEAV_jclass@@PEAU_jmethodID@@ZZ 0000000180001000 f i libsetenvstor001.obj
 0001:00000024       ?SetEventNotificationMode@_jvmtiEnv@@QEAA?AW4jvmtiError@@W4jvmtiEventMode@@W4jvmtiEvent@@PEAV_jobject@@ZZ 0000000180001024 f i libsetenvstor001.obj
 0001:0000002c       ?TranslateError@@YAPEBDW4jvmtiError@@@Z 000000018000102c f   libsetenvstor001.obj
 0001:000002e4       ?nsk_jni_check_exception@@YAHPEAUJNIEnv_@@QEBDH@Z 00000001800012e4 f   libsetenvstor001.obj
 0001:00000428       ?nsk_jni_lverify@@YAHHPEAUJNIEnv_@@HQEBDH1ZZ 0000000180001428 f   libsetenvstor001.obj
 0001:000004c8       Agent_Initialize           00000001800014c8 f   libsetenvstor001.obj
 0001:000007c8       Agent_OnAttach             00000001800017c8 f   libsetenvstor001.obj
 0001:000007c8       Agent_OnLoad               00000001800017c8 f   libsetenvstor001.obj
 0001:000007d0       Java_nsk_jvmti_unit_FollowReferences_FollowRefObjects_addRefToVerify 00000001800017d0 f   libsetenvstor001.obj
 0001:0000098c       Java_nsk_jvmti_unit_FollowReferences_FollowRefObjects_getTag 000000018000198c f   libsetenvstor001.obj
 0001:00000a48       Java_nsk_jvmti_unit_FollowReferences_FollowRefObjects_resetRefsToVerify 0000000180001a48 f   libsetenvstor001.obj
 0001:00000a50       Java_nsk_jvmti_unit_FollowReferences_FollowRefObjects_resetTags 0000000180001a50 f   libsetenvstor001.obj
 0001:00000a94       Java_nsk_jvmti_unit_FollowReferences_FollowRefObjects_setTag 0000000180001a94 f   libsetenvstor001.obj
 0001:00000ce0       Java_nsk_share_jvmti_ArgumentHandler_getAgentOptionsString 0000000180001ce0 f   libsetenvstor001.obj
 0001:00000d8c       Java_nsk_share_jvmti_DebugeeClass_checkStatus 0000000180001d8c f   libsetenvstor001.obj
 0001:00000e14       Java_nsk_share_jvmti_DebugeeClass_resetAgentData 0000000180001e14 f   libsetenvstor001.obj
 0001:00000e74       Java_nsk_share_jvmti_RedefineAgent_agentStatus 0000000180001e74 f   libsetenvstor001.obj
 0001:00000e80       Java_nsk_share_jvmti_RedefineAgent_isRedefined 0000000180001e80 f   libsetenvstor001.obj
 0001:00000e8c       Java_nsk_share_jvmti_RedefineAgent_redefineAttempted 0000000180001e8c f   libsetenvstor001.obj
 0001:00000e98       MA_checkStatus             0000000180001e98 f   libsetenvstor001.obj
 0001:00000f3c       __local_stdio_printf_options 0000000180001f3c f i libsetenvstor001.obj
 0001:0000119c       callbackVMDeath            000000018000219c f   libsetenvstor001.obj
 0001:00001278       callbackVMInit             0000000180002278 f   libsetenvstor001.obj
 0001:000015d0       exitOnError                00000001800025d0 f   libsetenvstor001.obj
 0001:00001684       fprintf                    0000000180002684 f i libsetenvstor001.obj
 0001:000016c8       nsk_complain               00000001800026c8 f   libsetenvstor001.obj
 0001:000016f4       nsk_jvmti_createJVMTIEnv   00000001800026f4 f   libsetenvstor001.obj
 0001:00001824       nsk_jvmti_enableEvents     0000000180002824 f   libsetenvstor001.obj
 0001:00001900       nsk_jvmti_lverify          0000000180002900 f   libsetenvstor001.obj
 0001:000019f0       nsk_jvmti_parseOptions     00000001800029f0 f   libsetenvstor001.obj
 0001:00001c40       nsk_jvmti_resetAgentData   0000000180002c40 f   libsetenvstor001.obj
 0001:00001cb4       nsk_jvmti_resumeSync       0000000180002cb4 f   libsetenvstor001.obj
 0001:00001d58       nsk_jvmti_waitForSync      0000000180002d58 f   libsetenvstor001.obj
 0001:00001e5c       nsk_lcomplain              0000000180002e5c f   libsetenvstor001.obj
 0001:00001e7c       nsk_ldisplay               0000000180002e7c f   libsetenvstor001.obj
 0001:00001e9c       nsk_ltrace                 0000000180002e9c f   libsetenvstor001.obj
 0001:00001ebc       nsk_lvcomplain             0000000180002ebc f   libsetenvstor001.obj
 0001:00002074       nsk_lvdisplay              0000000180003074 f   libsetenvstor001.obj
 0001:000020c0       nsk_lverify                00000001800030c0 f   libsetenvstor001.obj
 0001:0000211c       nsk_lvtrace                000000018000311c f   libsetenvstor001.obj
 0001:0000217c       nsk_printf                 000000018000317c f   libsetenvstor001.obj
 0001:000021a4       nsk_vprintf                00000001800031a4 f   libsetenvstor001.obj
 0001:00002258       printf                     0000000180003258 f i libsetenvstor001.obj
 0001:00002828       __raise_securityfailure    0000000180003828 f   MSVCRT:gs_report.obj
 0001:0000285c       __report_gsfailure         000000018000385c f   MSVCRT:gs_report.obj
 0001:00002a9c       __GSHandlerCheck           0000000180003a9c f   MSVCRT:gshandler.obj
 0001:00002abc       __GSHandlerCheckCommon     0000000180003abc f   MSVCRT:gshandler.obj
 0001:00002b30       __security_check_cookie    0000000180003b30 f   MSVCRT:amdsecgs.obj
 0001:00002e70       _DllMainCRTStartup         0000000180003e70 f   MSVCRT:dll_dllmain.obj
 0001:00002eb0       __scrt_acquire_startup_lock 0000000180003eb0 f   MSVCRT:utility.obj
 0001:00002eec       __scrt_dllmain_after_initialize_c 0000000180003eec f   MSVCRT:utility.obj
 0001:00002f20       __scrt_dllmain_before_initialize_c 0000000180003f20 f   MSVCRT:utility.obj
 0001:00002f38       __scrt_dllmain_crt_thread_attach 0000000180003f38 f   MSVCRT:utility.obj
 0001:00002f60       __scrt_dllmain_crt_thread_detach 0000000180003f60 f   MSVCRT:utility.obj
 0001:00002f78       __scrt_dllmain_exception_filter 0000000180003f78 f   MSVCRT:utility.obj
 0001:00002fd8       __scrt_dllmain_uninitialize_c 0000000180003fd8 f   MSVCRT:utility.obj
 0001:00003008       __scrt_dllmain_uninitialize_critical 0000000180004008 f   MSVCRT:utility.obj
 0001:0000301c       __scrt_initialize_crt      000000018000401c f   MSVCRT:utility.obj
 0001:00003068       __scrt_initialize_onexit_tables 0000000180004068 f   MSVCRT:utility.obj
 0001:000030f4       __scrt_is_nonwritable_in_current_image 00000001800040f4 f   MSVCRT:utility.obj
 0001:0000318c       __scrt_release_startup_lock 000000018000418c f   MSVCRT:utility.obj
 0001:000031b0       __scrt_uninitialize_crt    00000001800041b0 f   MSVCRT:utility.obj
 0001:000031dc       _onexit                    00000001800041dc f   MSVCRT:utility.obj
 0001:00003218       atexit                     0000000180004218 f   MSVCRT:utility.obj
 0001:00003230       __crt_debugger_hook        0000000180004230 f   MSVCRT:utility_desktop.obj
 0001:00003238       __scrt_fastfail            0000000180004238 f   MSVCRT:utility_desktop.obj
 0001:00003384       _guard_check_icall_nop     0000000180004384 f i MSVCRT:guard_support.obj
 0001:00003388       __security_init_cookie     0000000180004388 f   MSVCRT:gs_support.obj
 0001:00003434       DllMain                    0000000180004434 f   MSVCRT:dll_dllmain_stub.obj
 0001:00003458       ?__scrt_initialize_type_info@@YAXXZ 0000000180004458 f   MSVCRT:tncleanup.obj
 0001:00003468       ?__scrt_uninitialize_type_info@@YAXXZ 0000000180004468 f   MSVCRT:tncleanup.obj
 0001:00003474       __local_stdio_scanf_options 0000000180004474 f i MSVCRT:default_local_stdio_options.obj
 0001:0000347c       __scrt_initialize_default_local_stdio_options 000000018000447c f   MSVCRT:default_local_stdio_options.obj
 0001:00003498       __scrt_get_dyn_tls_init_callback 0000000180004498 f   MSVCRT:dyn_tls_init.obj
 0001:000034a0       _RTC_Initialize            00000001800044a0 f   MSVCRT:initsect.obj
 0001:000034dc       _RTC_Terminate             00000001800044dc f   MSVCRT:initsect.obj
 0001:00003518       __isa_available_init       0000000180004518 f   MSVCRT:cpu_disp.obj
 0001:000036c4       _get_startup_argv_mode     00000001800046c4 f   MSVCRT:argv_mode.obj
 0001:000036cc       __scrt_is_ucrt_dll_in_use  00000001800046cc f   MSVCRT:ucrt_detection.obj
 0001:000036e0       memcpy                     00000001800046e0 f   vcruntime:VCRUNTIME140.dll
 0001:000036e6       memset                     00000001800046e6 f   vcruntime:VCRUNTIME140.dll
 0001:000036ec       strchr                     00000001800046ec f   vcruntime:VCRUNTIME140.dll
 0001:000036f2       __C_specific_handler       00000001800046f2 f   vcruntime:VCRUNTIME140.dll
 0001:000036f8       __std_type_info_destroy_list 00000001800046f8 f   vcruntime:VCRUNTIME140.dll
 0001:000036fe       strcmp                     00000001800046fe f   ucrt:api-ms-win-crt-string-l1-1-0.dll
 0001:00003704       strlen                     0000000180004704 f   ucrt:api-ms-win-crt-string-l1-1-0.dll
 0001:0000370a       _initterm                  000000018000470a f   ucrt:api-ms-win-crt-runtime-l1-1-0.dll
 0001:00003710       _initterm_e                0000000180004710 f   ucrt:api-ms-win-crt-runtime-l1-1-0.dll
 0001:00003716       _seh_filter_dll            0000000180004716 f   ucrt:api-ms-win-crt-runtime-l1-1-0.dll
 0001:0000371c       _configure_narrow_argv     000000018000471c f   ucrt:api-ms-win-crt-runtime-l1-1-0.dll
 0001:00003722       _initialize_narrow_environment 0000000180004722 f   ucrt:api-ms-win-crt-runtime-l1-1-0.dll
 0001:00003728       _initialize_onexit_table   0000000180004728 f   ucrt:api-ms-win-crt-runtime-l1-1-0.dll
 0001:0000372e       _register_onexit_function  000000018000472e f   ucrt:api-ms-win-crt-runtime-l1-1-0.dll
 0001:00003734       _execute_onexit_table      0000000180004734 f   ucrt:api-ms-win-crt-runtime-l1-1-0.dll
 0001:0000373a       _crt_atexit                000000018000473a f   ucrt:api-ms-win-crt-runtime-l1-1-0.dll
 0001:00003740       _cexit                     0000000180004740 f   ucrt:api-ms-win-crt-runtime-l1-1-0.dll
 0001:00003748       __acrt_initialize          0000000180004748 f   MSVCRT:ucrt_stubs.obj
 0001:00003748       __acrt_thread_attach       0000000180004748 f   MSVCRT:ucrt_stubs.obj
 0001:00003748       __acrt_thread_detach       0000000180004748 f   MSVCRT:ucrt_stubs.obj
 0001:00003748       __acrt_uninitialize        0000000180004748 f   MSVCRT:ucrt_stubs.obj
 0001:00003748       __acrt_uninitialize_critical 0000000180004748 f   MSVCRT:ucrt_stubs.obj
 0001:00003748       __scrt_stub_for_acrt_initialize 0000000180004748 f   MSVCRT:ucrt_stubs.obj
 0001:00003748       __scrt_stub_for_acrt_thread_attach 0000000180004748 f   MSVCRT:ucrt_stubs.obj
 0001:00003748       __scrt_stub_for_acrt_thread_detach 0000000180004748 f   MSVCRT:ucrt_stubs.obj
 0001:00003748       __scrt_stub_for_acrt_uninitialize 0000000180004748 f   MSVCRT:ucrt_stubs.obj
 0001:00003748       __scrt_stub_for_acrt_uninitialize_critical 0000000180004748 f   MSVCRT:ucrt_stubs.obj
 0001:00003748       __vcrt_initialize          0000000180004748 f   MSVCRT:ucrt_stubs.obj
 0001:00003748       __vcrt_thread_attach       0000000180004748 f   MSVCRT:ucrt_stubs.obj
 0001:00003748       __vcrt_thread_detach       0000000180004748 f   MSVCRT:ucrt_stubs.obj
 0001:00003748       __vcrt_uninitialize        0000000180004748 f   MSVCRT:ucrt_stubs.obj
 0001:00003748       __vcrt_uninitialize_critical 0000000180004748 f   MSVCRT:ucrt_stubs.obj
 0001:0000374c       __scrt_stub_for_is_c_termination_complete 000000018000474c f   MSVCRT:ucrt_stubs.obj
 0001:0000374c       _is_c_termination_complete 000000018000474c f   MSVCRT:ucrt_stubs.obj
 0001:00003760       _guard_dispatch_icall_nop  0000000180004760 f   MSVCRT:guard_dispatch.obj
 0001:00003780       _guard_xfg_dispatch_icall_nop 0000000180004780 f   MSVCRT:guard_xfg_dispatch.obj
 0002:00000000       __imp_RtlCaptureContext    0000000180005000     kernel32:KERNEL32.dll
 0002:00000008       __imp_RtlLookupFunctionEntry 0000000180005008     kernel32:KERNEL32.dll
 0002:00000010       __imp_RtlVirtualUnwind     0000000180005010     kernel32:KERNEL32.dll
 0002:00000018       __imp_UnhandledExceptionFilter 0000000180005018     kernel32:KERNEL32.dll
 0002:00000020       __imp_SetUnhandledExceptionFilter 0000000180005020     kernel32:KERNEL32.dll
 0002:00000028       __imp_GetCurrentProcess    0000000180005028     kernel32:KERNEL32.dll
 0002:00000030       __imp_TerminateProcess     0000000180005030     kernel32:KERNEL32.dll
 0002:00000038       __imp_IsProcessorFeaturePresent 0000000180005038     kernel32:KERNEL32.dll
 0002:00000040       __imp_CloseHandle          0000000180005040     kernel32:KERNEL32.dll
 0002:00000048       __imp_InitializeCriticalSectionAndSpinCount 0000000180005048     kernel32:KERNEL32.dll
 0002:00000050       __imp_DeleteCriticalSection 0000000180005050     kernel32:KERNEL32.dll
 0002:00000058       __imp_CreateEventW         0000000180005058     kernel32:KERNEL32.dll
 0002:00000060       __imp_GetModuleHandleW     0000000180005060     kernel32:KERNEL32.dll
 0002:00000068       __imp_GetProcAddress       0000000180005068     kernel32:KERNEL32.dll
 0002:00000070       __imp_IsDebuggerPresent    0000000180005070     kernel32:KERNEL32.dll
 0002:00000078       __imp_QueryPerformanceCounter 0000000180005078     kernel32:KERNEL32.dll
 0002:00000080       __imp_GetCurrentProcessId  0000000180005080     kernel32:KERNEL32.dll
 0002:00000088       __imp_GetCurrentThreadId   0000000180005088     kernel32:KERNEL32.dll
 0002:00000090       __imp_GetSystemTimeAsFileTime 0000000180005090     kernel32:KERNEL32.dll
 0002:00000098       __imp_DisableThreadLibraryCalls 0000000180005098     kernel32:KERNEL32.dll
 0002:000000a0       __imp_InitializeSListHead  00000001800050a0     kernel32:KERNEL32.dll
 0002:000000a8       \177KERNEL32_NULL_THUNK_DATA 00000001800050a8     kernel32:KERNEL32.dll
 0002:000000b0       __imp_memcpy               00000001800050b0     vcruntime:VCRUNTIME140.dll
 0002:000000b8       __imp_memset               00000001800050b8     vcruntime:VCRUNTIME140.dll
 0002:000000c0       __imp_strchr               00000001800050c0     vcruntime:VCRUNTIME140.dll
 0002:000000c8       __imp___C_specific_handler 00000001800050c8     vcruntime:VCRUNTIME140.dll
 0002:000000d0       __imp___std_type_info_destroy_list 00000001800050d0     vcruntime:VCRUNTIME140.dll
 0002:000000d8       \177VCRUNTIME140_NULL_THUNK_DATA 00000001800050d8     vcruntime:VCRUNTIME140.dll
 0002:000000e0       __imp_strtol               00000001800050e0     ucrt:api-ms-win-crt-convert-l1-1-0.dll
 0002:000000e8       \177api-ms-win-crt-convert-l1-1-0_NULL_THUNK_DATA 00000001800050e8     ucrt:api-ms-win-crt-convert-l1-1-0.dll
 0002:000000f0       __imp_malloc               00000001800050f0     ucrt:api-ms-win-crt-heap-l1-1-0.dll
 0002:000000f8       __imp_free                 00000001800050f8     ucrt:api-ms-win-crt-heap-l1-1-0.dll
 0002:00000100       \177api-ms-win-crt-heap-l1-1-0_NULL_THUNK_DATA 0000000180005100     ucrt:api-ms-win-crt-heap-l1-1-0.dll
 0002:00000108       __imp__errno               0000000180005108     ucrt:api-ms-win-crt-runtime-l1-1-0.dll
 0002:00000110       __imp_exit                 0000000180005110     ucrt:api-ms-win-crt-runtime-l1-1-0.dll
 0002:00000118       __imp__cexit               0000000180005118     ucrt:api-ms-win-crt-runtime-l1-1-0.dll
 0002:00000120       __imp__crt_atexit          0000000180005120     ucrt:api-ms-win-crt-runtime-l1-1-0.dll
 0002:00000128       __imp__execute_onexit_table 0000000180005128     ucrt:api-ms-win-crt-runtime-l1-1-0.dll
 0002:00000130       __imp__register_onexit_function 0000000180005130     ucrt:api-ms-win-crt-runtime-l1-1-0.dll
 0002:00000138       __imp__initialize_onexit_table 0000000180005138     ucrt:api-ms-win-crt-runtime-l1-1-0.dll
 0002:00000140       __imp__initialize_narrow_environment 0000000180005140     ucrt:api-ms-win-crt-runtime-l1-1-0.dll
 0002:00000148       __imp__configure_narrow_argv 0000000180005148     ucrt:api-ms-win-crt-runtime-l1-1-0.dll
 0002:00000150       __imp__seh_filter_dll      0000000180005150     ucrt:api-ms-win-crt-runtime-l1-1-0.dll
 0002:00000158       __imp__initterm_e          0000000180005158     ucrt:api-ms-win-crt-runtime-l1-1-0.dll
 0002:00000160       __imp__initterm            0000000180005160     ucrt:api-ms-win-crt-runtime-l1-1-0.dll
 0002:00000168       \177api-ms-win-crt-runtime-l1-1-0_NULL_THUNK_DATA 0000000180005168     ucrt:api-ms-win-crt-runtime-l1-1-0.dll
 0002:00000170       __imp___acrt_iob_func      0000000180005170     ucrt:api-ms-win-crt-stdio-l1-1-0.dll
 0002:00000178       __imp_fflush               0000000180005178     ucrt:api-ms-win-crt-stdio-l1-1-0.dll
 0002:00000180       __imp___stdio_common_vsprintf 0000000180005180     ucrt:api-ms-win-crt-stdio-l1-1-0.dll
 0002:00000188       __imp___stdio_common_vfprintf 0000000180005188     ucrt:api-ms-win-crt-stdio-l1-1-0.dll
 0002:00000190       \177api-ms-win-crt-stdio-l1-1-0_NULL_THUNK_DATA 0000000180005190     ucrt:api-ms-win-crt-stdio-l1-1-0.dll
 0002:00000198       __imp_strcmp               0000000180005198     ucrt:api-ms-win-crt-string-l1-1-0.dll
 0002:000001a0       __imp__strdup              00000001800051a0     ucrt:api-ms-win-crt-string-l1-1-0.dll
 0002:000001a0       __imp_strdup               00000001800051a0     ucrt:api-ms-win-crt-string-l1-1-0.dll
 0002:000001a8       __imp_strlen               00000001800051a8     ucrt:api-ms-win-crt-string-l1-1-0.dll
 0002:000001b0       __imp_strpbrk              00000001800051b0     ucrt:api-ms-win-crt-string-l1-1-0.dll
 0002:000001b8       __imp_strncpy              00000001800051b8     ucrt:api-ms-win-crt-string-l1-1-0.dll
 0002:000001c0       \177api-ms-win-crt-string-l1-1-0_NULL_THUNK_DATA 00000001800051c0     ucrt:api-ms-win-crt-string-l1-1-0.dll
 0002:000001c8       __guard_check_icall_fptr   00000001800051c8     MSVCRT:guard_support.obj
 0002:000001d0       __guard_xfg_check_icall_fptr 00000001800051d0     MSVCRT:guard_support.obj
 0002:000001d8       __guard_dispatch_icall_fptr 00000001800051d8     MSVCRT:guard_support.obj
 0002:000001e0       __guard_xfg_dispatch_icall_fptr 00000001800051e0     MSVCRT:guard_support.obj
 0002:000001e8       __guard_xfg_table_dispatch_icall_fptr 00000001800051e8     MSVCRT:guard_support.obj
 0002:000001f0       __castguard_check_failure_os_handled_fptr 00000001800051f0     MSVCRT:guard_support.obj
 0002:000001f8       __guard_memcpy_fptr        00000001800051f8     vcruntime:softmemtag.obj
 0002:00000200       __xc_a                     0000000180005200     MSVCRT:initializers.obj
 0002:00000208       __xc_z                     0000000180005208     MSVCRT:initializers.obj
 0002:00000210       __xi_a                     0000000180005210     MSVCRT:initializers.obj
 0002:00000220       __xi_z                     0000000180005220     MSVCRT:initializers.obj
 0002:00000228       __xl_a                     0000000180005228     MSVCRT:tlssup.obj
 0002:00000230       __xl_z                     0000000180005230     MSVCRT:tlssup.obj
 0002:00000238       __xp_a                     0000000180005238     MSVCRT:initializers.obj
 0002:00000240       __xp_z                     0000000180005240     MSVCRT:initializers.obj
 0002:00000248       __xt_a                     0000000180005248     MSVCRT:initializers.obj
 0002:00000250       __xt_z                     0000000180005250     MSVCRT:initializers.obj
 0002:00000260       g_refKindStr               0000000180005260     libsetenvstor001.obj
 0002:00000410       ??_C@_09BPLDFGCI@unknown_0@ 0000000180005410     libsetenvstor001.obj
 0002:00000420       ??_C@_0BL@FPNMECJD@JVMTI_HEAP_REFERENCE_CLASS@ 0000000180005420     libsetenvstor001.obj
 0002:00000440       ??_C@_0BL@FKGKKLNM@JVMTI_HEAP_REFERENCE_FIELD@ 0000000180005440     libsetenvstor001.obj
 0002:00000460       ??_C@_0CD@CAEHCFJF@JVMTI_HEAP_REFERENCE_ARRAY_ELEM@ 0000000180005460     libsetenvstor001.obj
 0002:00000488       ??_C@_0CC@DNEBMCNK@JVMTI_HEAP_REFERENCE_CLASS_LOAD@ 0000000180005488     libsetenvstor001.obj
 0002:000004b0       ??_C@_0BN@CJMIPEBB@JVMTI_HEAP_REFERENCE_SIGNERS@ 00000001800054b0     libsetenvstor001.obj
 0002:000004d0       ??_C@_0CH@HBOIDPEB@JVMTI_HEAP_REFERENCE_PROTECTION@ 00000001800054d0     libsetenvstor001.obj
 0002:000004f8       ??_C@_0BP@MDKGDGKL@JVMTI_HEAP_REFERENCE_INTERFACE@ 00000001800054f8     libsetenvstor001.obj
 0002:00000518       ??_C@_0CC@JJMIHNJH@JVMTI_HEAP_REFERENCE_STATIC_FIE@ 0000000180005518     libsetenvstor001.obj
 0002:00000540       ??_C@_0CD@IDHEEGID@JVMTI_HEAP_REFERENCE_CONSTANT_P@ 0000000180005540     libsetenvstor001.obj
 0002:00000568       ??_C@_0CA@EFFCHNG@JVMTI_HEAP_REFERENCE_SUPERCLASS@ 0000000180005568     libsetenvstor001.obj
 0002:00000588       ??_C@_0L@PCDFHGCJ@unknown_11@ 0000000180005588     libsetenvstor001.obj
 0002:00000598       ??_C@_0L@NJBICFOK@unknown_12@ 0000000180005598     libsetenvstor001.obj
 0002:000005a8       ??_C@_0L@MAADBEKL@unknown_13@ 00000001800055a8     libsetenvstor001.obj
 0002:000005b8       ??_C@_0L@IPECICGM@unknown_14@ 00000001800055b8     libsetenvstor001.obj
 0002:000005c8       ??_C@_0L@JGFJLDCN@unknown_15@ 00000001800055c8     libsetenvstor001.obj
 0002:000005d8       ??_C@_0L@LNHEOAOO@unknown_16@ 00000001800055d8     libsetenvstor001.obj
 0002:000005e8       ??_C@_0L@KEGPNBKP@unknown_17@ 00000001800055e8     libsetenvstor001.obj
 0002:000005f8       ??_C@_0L@CDPHMNGA@unknown_18@ 00000001800055f8     libsetenvstor001.obj
 0002:00000608       ??_C@_0L@DKOMPMCB@unknown_19@ 0000000180005608     libsetenvstor001.obj
 0002:00000618       ??_C@_0L@OJGIPJDB@unknown_20@ 0000000180005618     libsetenvstor001.obj
 0002:00000628       ??_C@_0CA@KAOFNDEM@JVMTI_HEAP_REFERENCE_JNI_GLOBAL@ 0000000180005628     libsetenvstor001.obj
 0002:00000648       ??_C@_0CC@HPFAJBK@JVMTI_HEAP_REFERENCE_SYSTEM_CLA@ 0000000180005648     libsetenvstor001.obj
 0002:00000670       ??_C@_0BN@FDEGFOHC@JVMTI_HEAP_REFERENCE_MONITOR@ 0000000180005670     libsetenvstor001.obj
 0002:00000690       ??_C@_0CB@HKIBCMAJ@JVMTI_HEAP_REFERENCE_STACK_LOCA@ 0000000180005690     libsetenvstor001.obj
 0002:000006b8       ??_C@_0BP@EAACMMOE@JVMTI_HEAP_REFERENCE_JNI_LOCAL@ 00000001800056b8     libsetenvstor001.obj
 0002:000006d8       ??_C@_0BM@IJDEOGOE@JVMTI_HEAP_REFERENCE_THREAD@ 00000001800056d8     libsetenvstor001.obj
 0002:000006f8       ??_C@_0BL@EDGPPKC@JVMTI_HEAP_REFERENCE_OTHER@ 00000001800056f8     libsetenvstor001.obj
 0002:00000714       ??_C@_04BCJPDBDA@Code@     0000000180005714     libsetenvstor001.obj
 0002:00000720       ??_C@_0BA@OCLMCFKC@LineNumberTable@ 0000000180005720     libsetenvstor001.obj
 0002:00000730       ??_C@_0BD@CPAEPILC@LocalVariableTable@ 0000000180005730     libsetenvstor001.obj
 0002:00000748       ??_C@_0BH@NMBDNHBD@LocalVariableTypeTable@ 0000000180005748     libsetenvstor001.obj
 0002:00000760       ??_C@_0O@HIHEEDNJ@StackMapTable@ 0000000180005760     libsetenvstor001.obj
 0002:00000770       ??_C@_0L@HCDIAMJG@?9?5?$CFs?0?5?$CFd?3?5@ 0000000180005770     libsetenvstor001.obj
 0002:00000780       ??_C@_0JI@HLPECLFI@?$CD?5?4?4?4?6?$CD?5ERROR?3?5too?5many?5complai@ 0000000180005780     libsetenvstor001.obj
 0002:00000820       ??_C@_0ED@JNEKCCOB@The?5following?5fake?5exception?5st@ 0000000180005820     libsetenvstor001.obj
 0002:00000868       ??_C@_0CN@FCNMDFBH@nsk?4share?4Fake_Exception_for_RU@ 0000000180005868     libsetenvstor001.obj
 0002:00000898       ??_C@_08PGFFNAEI@?$CI?$CFs?3?$CFd?$CJ?5@ 0000000180005898     libsetenvstor001.obj
 0002:000008a8       ??_C@_0DP@IENMAEGI@s?2test?2hotspot?2jtreg?2vmTestbase@ 00000001800058a8     libsetenvstor001.obj
 0002:000008e8       ??_C@_0BL@NDJLFFJB@?7at?5nsk_lvcomplain?$CI?$CFs?3?$CFd?$CJ?6@ 00000001800058e8     libsetenvstor001.obj
 0002:00000908       ??_C@_0BC@JOOKAFKF@?$CD?5ERROR?3?5?$CFs?0?5?$CFd?3?5@ 0000000180005908     libsetenvstor001.obj
 0002:00000920       ??_C@_09KJEAHMEH@?$CD?5ERROR?3?5@ 0000000180005920     libsetenvstor001.obj
 0002:0000092c       ??_C@_02GPIOPFAK@?$DO?$DO@ 000000018000592c     libsetenvstor001.obj
 0002:00000930       ??_C@_02FODMEDOG@?$DM?$DM@ 0000000180005930     libsetenvstor001.obj
 0002:00000934       ??_C@_02DJGKEECL@?4?4@     0000000180005934     libsetenvstor001.obj
 0002:00000938       ??_C@_0O@CJPGJOAF@?9?5?$CFs?0?5?$CFd?3?5?$CFs?5@ 0000000180005938     libsetenvstor001.obj
 0002:00000948       ??_C@_0CB@IAKPDOIC@?$CD?5?5?5verified?5assertion?5is?5FALSE@ 0000000180005948     libsetenvstor001.obj
 0002:00000970       ??_C@_0CO@LGONDEPD@stdout?3?5fflush?5failed?5?9?5err?$DN?$CFd?5@ 0000000180005970     libsetenvstor001.obj
 0002:000009a0       ??_C@_0CO@KBGKJPBD@stderr?3?5fflush?5failed?5?9?5err?$DN?$CFd?5@ 00000001800059a0     libsetenvstor001.obj
 0002:000009d0       ??_C@_0BB@JCNMKLLK@JVMTI_ERROR_NONE@ 00000001800059d0     libsetenvstor001.obj
 0002:000009e8       ??_C@_0BL@LDIMKLPH@JVMTI_ERROR_INVALID_THREAD@ 00000001800059e8     libsetenvstor001.obj
 0002:00000a08       ??_C@_0CB@PJFPAIKJ@JVMTI_ERROR_INVALID_THREAD_GROU@ 0000000180005a08     libsetenvstor001.obj
 0002:00000a30       ??_C@_0BN@LLMKHMNF@JVMTI_ERROR_INVALID_PRIORITY@ 0000000180005a30     libsetenvstor001.obj
 0002:00000a50       ??_C@_0CB@MBOFKAGB@JVMTI_ERROR_THREAD_NOT_SUSPENDE@ 0000000180005a50     libsetenvstor001.obj
 0002:00000a78       ??_C@_0BN@FABOLPBI@JVMTI_ERROR_THREAD_SUSPENDED@ 0000000180005a78     libsetenvstor001.obj
 0002:00000a98       ??_C@_0BN@FDGNOBJM@JVMTI_ERROR_THREAD_NOT_ALIVE@ 0000000180005a98     libsetenvstor001.obj
 0002:00000ab8       ??_C@_0BL@GOBIFKNJ@JVMTI_ERROR_INVALID_OBJECT@ 0000000180005ab8     libsetenvstor001.obj
 0002:00000ad8       ??_C@_0BK@FCMAJPPC@JVMTI_ERROR_INVALID_CLASS@ 0000000180005ad8     libsetenvstor001.obj
 0002:00000af8       ??_C@_0BP@IKLLBKEB@JVMTI_ERROR_CLASS_NOT_PREPARED@ 0000000180005af8     libsetenvstor001.obj
 0002:00000b18       ??_C@_0BN@KLPPLKG@JVMTI_ERROR_INVALID_METHODID@ 0000000180005b18     libsetenvstor001.obj
 0002:00000b38       ??_C@_0BN@BCEKOKND@JVMTI_ERROR_INVALID_LOCATION@ 0000000180005b38     libsetenvstor001.obj
 0002:00000b58       ??_C@_0BM@DFDGPME@JVMTI_ERROR_INVALID_FIELDID@ 0000000180005b58     libsetenvstor001.obj
 0002:00000b78       ??_C@_0BL@NELIEPEC@JVMTI_ERROR_NO_MORE_FRAMES@ 0000000180005b78     libsetenvstor001.obj
 0002:00000b98       ??_C@_0BJ@BDBECFDM@JVMTI_ERROR_OPAQUE_FRAME@ 0000000180005b98     libsetenvstor001.obj
 0002:00000bb8       ??_C@_0BK@MIIFNLOB@JVMTI_ERROR_TYPE_MISMATCH@ 0000000180005bb8     libsetenvstor001.obj
 0002:00000bd8       ??_C@_0BJ@HPCAOILC@JVMTI_ERROR_INVALID_SLOT@ 0000000180005bd8     libsetenvstor001.obj
 0002:00000bf8       ??_C@_0BG@CHILOPNI@JVMTI_ERROR_DUPLICATE@ 0000000180005bf8     libsetenvstor001.obj
 0002:00000c10       ??_C@_0BG@DIEMLHKM@JVMTI_ERROR_NOT_FOUND@ 0000000180005c10     libsetenvstor001.obj
 0002:00000c28       ??_C@_0BM@NHMCKHOB@JVMTI_ERROR_INVALID_MONITOR@ 0000000180005c28     libsetenvstor001.obj
 0002:00000c48       ??_C@_0BO@PPEDAJGL@JVMTI_ERROR_NOT_MONITOR_OWNER@ 0000000180005c48     libsetenvstor001.obj
 0002:00000c68       ??_C@_0BG@FCAIPEID@JVMTI_ERROR_INTERRUPT@ 0000000180005c68     libsetenvstor001.obj
 0002:00000c80       ??_C@_0CB@EGDBNKOI@JVMTI_ERROR_INVALID_CLASS_FORMA@ 0000000180005c80     libsetenvstor001.obj
 0002:00000ca8       ??_C@_0CG@DGKOGIAL@JVMTI_ERROR_CIRCULAR_CLASS_DEFI@ 0000000180005ca8     libsetenvstor001.obj
 0002:00000cd0       ??_C@_0BP@ICEALPKC@JVMTI_ERROR_FAILS_VERIFICATION@ 0000000180005cd0     libsetenvstor001.obj
 0002:00000cf0       ??_C@_0DC@JDACLMIO@JVMTI_ERROR_UNSUPPORTED_REDEFIN@ 0000000180005cf0     libsetenvstor001.obj
 0002:00000d28       ??_C@_0DE@GKDKNOMJ@JVMTI_ERROR_UNSUPPORTED_REDEFIN@ 0000000180005d28     libsetenvstor001.obj
 0002:00000d60       ??_C@_0BO@LAFKIOG@JVMTI_ERROR_INVALID_TYPESTATE@ 0000000180005d60     libsetenvstor001.obj
 0002:00000d80       ??_C@_0DH@INDGCLLB@JVMTI_ERROR_UNSUPPORTED_REDEFIN@ 0000000180005d80     libsetenvstor001.obj
 0002:00000db8       ??_C@_0DE@NHEOMMGI@JVMTI_ERROR_UNSUPPORTED_REDEFIN@ 0000000180005db8     libsetenvstor001.obj
 0002:00000df0       ??_C@_0CA@EKPNJOEP@JVMTI_ERROR_UNSUPPORTED_VERSION@ 0000000180005df0     libsetenvstor001.obj
 0002:00000e10       ??_C@_0BN@OFFMAHHL@JVMTI_ERROR_NAMES_DONT_MATCH@ 0000000180005e10     libsetenvstor001.obj
 0002:00000e30       ??_C@_0DN@HHBBLAKE@JVMTI_ERROR_UNSUPPORTED_REDEFIN@ 0000000180005e30     libsetenvstor001.obj
 0002:00000e70       ??_C@_0DO@HMBGBGNA@JVMTI_ERROR_UNSUPPORTED_REDEFIN@ 0000000180005e70     libsetenvstor001.obj
 0002:00000eb0       ??_C@_0BP@PBECGKHJ@JVMTI_ERROR_UNMODIFIABLE_CLASS@ 0000000180005eb0     libsetenvstor001.obj
 0002:00000ed0       ??_C@_0BK@CANILEHF@JVMTI_ERROR_NOT_AVAILABLE@ 0000000180005ed0     libsetenvstor001.obj
 0002:00000ef0       ??_C@_0CE@INJKMEFK@JVMTI_ERROR_MUST_POSSESS_CAPABI@ 0000000180005ef0     libsetenvstor001.obj
 0002:00000f18       ??_C@_0BJ@LBFPFPDM@JVMTI_ERROR_NULL_POINTER@ 0000000180005f18     libsetenvstor001.obj
 0002:00000f38       ??_C@_0BP@CHJPNNEM@JVMTI_ERROR_ABSENT_INFORMATION@ 0000000180005f38     libsetenvstor001.obj
 0002:00000f58       ??_C@_0BP@OMFMNLC@JVMTI_ERROR_INVALID_EVENT_TYPE@ 0000000180005f58     libsetenvstor001.obj
 0002:00000f78       ??_C@_0BN@BIBNPHHO@JVMTI_ERROR_ILLEGAL_ARGUMENT@ 0000000180005f78     libsetenvstor001.obj
 0002:00000f98       ??_C@_0BK@KKNDHDCE@JVMTI_ERROR_NATIVE_METHOD@ 0000000180005f98     libsetenvstor001.obj
 0002:00000fb8       ??_C@_0BK@PMKCFHAE@JVMTI_ERROR_OUT_OF_MEMORY@ 0000000180005fb8     libsetenvstor001.obj
 0002:00000fd8       ??_C@_0BK@NNJBDMNB@JVMTI_ERROR_ACCESS_DENIED@ 0000000180005fd8     libsetenvstor001.obj
 0002:00000ff8       ??_C@_0BI@GHECLMNC@JVMTI_ERROR_WRONG_PHASE@ 0000000180005ff8     libsetenvstor001.obj
 0002:00001010       ??_C@_0BF@OLIHJOII@JVMTI_ERROR_INTERNAL@ 0000000180006010     libsetenvstor001.obj
 0002:00001028       ??_C@_0BO@EOHGKJHI@JVMTI_ERROR_UNATTACHED_THREAD@ 0000000180006028     libsetenvstor001.obj
 0002:00001048       ??_C@_0CA@LKHFDACL@JVMTI_ERROR_INVALID_ENVIRONMENT@ 0000000180006048     libsetenvstor001.obj
 0002:00001068       ??_C@_0BA@MMFHLOKK@?$DMunknown?5error?$DO@ 0000000180006068     libsetenvstor001.obj
 0002:00001078       ??_C@_0CF@CBHOKDB@throwable?5?$DN?5jni?9?$DOExceptionOccur@ 0000000180006078     libsetenvstor001.obj
 0002:000010a0       ??_C@_03OFAPEBGM@?$CFs?6@  00000001800060a0     libsetenvstor001.obj
 0002:000010a8       ??_C@_0DM@LPIGEGNJ@s?2test?2hotspot?2jtreg?2vmTestbase@ 00000001800060a8     libsetenvstor001.obj
 0002:000010e8       ??_C@_0CC@NFCNPEPK@Exception?5in?5JNI?5call?5?$CIcleared?$CJ@ 00000001800060e8     libsetenvstor001.obj
 0002:00001110       ??_C@_0BJ@IBAKFIKF@jni?9?$DOExceptionDescribe?$CI?$CJ@ 0000000180006110     libsetenvstor001.obj
 0002:00001130       ??_C@_0BG@GGKALKMH@jni?9?$DOExceptionClear?$CI?$CJ@ 0000000180006130     libsetenvstor001.obj
 0002:00001148       ??_C@_0CF@JMGFGJLJ@?$CD?5?5?5verified?5JNI?5assertion?5is?5F@ 0000000180006148     libsetenvstor001.obj
 0002:00001170       ??_C@_07KBAMPNJK@verbose@  0000000180006170     libsetenvstor001.obj
 0002:00001178       ??_C@_0DN@PKJBOLAP@nsk_jvmti_parseOptions?$CI?$CJ?3?5unexp@ 0000000180006178     libsetenvstor001.obj
 0002:000011b8       ??_C@_05IMBNNINJ@trace@    00000001800061b8     libsetenvstor001.obj
 0002:000011c0       ??_C@_0DD@BJKGNDMB@nsk_jvmti_parseOptions?$CI?$CJ?3?5no?5va@ 00000001800061c0     libsetenvstor001.obj
 0002:000011f4       ??_C@_04CGFJFPFD@none@     00000001800061f4     libsetenvstor001.obj
 0002:000011fc       ??_C@_06BMELKFMA@before@   00000001800061fc     libsetenvstor001.obj
 0002:00001204       ??_C@_05CMKPCFDK@after@    0000000180006204     libsetenvstor001.obj
 0002:0000120c       ??_C@_03NFKEKGGK@all@      000000018000620c     libsetenvstor001.obj
 0002:00001210       ??_C@_0DM@NDNJGJKE@nsk_jvmti_parseOptions?$CI?$CJ?3?5uexpe@ 0000000180006210     libsetenvstor001.obj
 0002:00001250       ??_C@_08NBBJKJO@waittime@  0000000180006250     libsetenvstor001.obj
 0002:00001260       ??_C@_0DO@CMHGAOHC@nsk_jvmti_parseOptions?$CI?$CJ?3?5not?5i@ 0000000180006260     libsetenvstor001.obj
 0002:000012a0       ??_C@_0DL@LNMPBDLN@nsk_jvmti_parseOptions?$CI?$CJ?3?5negat@ 00000001800062a0     libsetenvstor001.obj
 0002:000012e0       ??_C@_0DA@GMFJNOJH@nsk_jvmti_parseOptions?$CI?$CJ?3?5unkno@ 00000001800062e0     libsetenvstor001.obj
 0002:00001310       ??_C@_0CO@CCIAMEAN@nsk_jvmti_parseOptions?$CI?$CJ?3?5found@ 0000000180006310     libsetenvstor001.obj
 0002:00001340       ??_C@_0CJ@OEGPCGDL@nsk_jvmti_parseOptions?$CI?$CJ?3?5out?5o@ 0000000180006340     libsetenvstor001.obj
 0002:00001370       ??_C@_0DI@NMBHPGGF@nsk_jvmti_parseOptions?$CI?$CJ?3?5too?5m@ 0000000180006370     libsetenvstor001.obj
 0002:000013a8       ??_C@_03POGCGECB@?5?0?$HO@ 00000001800063a8     libsetenvstor001.obj
 0002:000013b0       ??_C@_0CB@MLNJNCLJ@?5?5jvmti?5error?3?5code?$DN?$CFd?0?5name?$DN?$CFs@ 00000001800063b0     libsetenvstor001.obj
 0002:000013d8       ??_C@_0CD@OHBGDKMK@?$CD?5?5?5jvmti?5error?3?5code?$DN?$CFd?0?5name?$DN@ 00000001800063d8     libsetenvstor001.obj
 0002:00001400       ??_C@_0CG@JNNCGPHB@?$CD?5?5?5error?5expected?3?5code?$DN?$CFd?0?5na@ 0000000180006400     libsetenvstor001.obj
 0002:00001430       ??_C@_0EB@IMGKPCGE@?$CIstr_obj?5?$DN?5jni?9?$DONewStringUTF?$CIco@ 0000000180006430     libsetenvstor001.obj
 0002:00001480       ??_C@_0EA@HFOGGBCC@s?2test?2hotspot?2jtreg?2vmTestbase@ 0000000180006480     libsetenvstor001.obj
 0002:000014c0       ??_C@_05KKCIMGE@error@     00000001800064c0     libsetenvstor001.obj
 0002:000014c8       ??_C@_0BD@HGNAOMCP@agent_data_monitor@ 00000001800064c8     libsetenvstor001.obj
 0002:000014e0       ??_C@_0EB@OGCLGKLN@javaVM?9?$DOGetEnv?$CI?$CIvoid?5?$CK?$CK?$CJ?$CGjvmti_@ 00000001800064e0     libsetenvstor001.obj
 0002:00001530       ??_C@_0EA@PNBCDMOA@s?2test?2hotspot?2jtreg?2vmTestbase@ 0000000180006530     libsetenvstor001.obj
 0002:00001570       ??_C@_0CI@DDPIFBGM@init_agent_data?$CIjvmti_env?0?5?$CGage@ 0000000180006570     libsetenvstor001.obj
 0002:00001598       ??_C@_0DI@ILAHDLMP@?$CI?$CKagentThreadProc?$CJ?$CIjvmti_env?0?5a@ 0000000180006598     libsetenvstor001.obj
 0002:000015d0       ??_C@_0BD@KDBALNLB@JVMTI?5agent?5thread@ 00000001800065d0     libsetenvstor001.obj
 0002:000015e8       ??_C@_0BB@NOKBFPFO@java?1lang?1Thread@ 00000001800065e8     libsetenvstor001.obj
 0002:000015fc       ??_C@_06FALKBLGB@?$DMinit?$DO@ 00000001800065fc     libsetenvstor001.obj
 0002:00001608       ??_C@_0BG@IKDDPPGD@?$CILjava?1lang?1String?$DL?$CJV@ 0000000180006608     libsetenvstor001.obj
 0002:00001620       ??_C@_0EB@IFJBFEKC@?$CIthreadClass?5?$DN?5jni_env?9?$DOFindCla@ 0000000180006620     libsetenvstor001.obj
 0002:00001670       ??_C@_0GF@FGFIBKKL@?$CIthreadCtor?5?$DN?5jni_env?9?$DOGetMetho@ 0000000180006670     libsetenvstor001.obj
 0002:000016d8       ??_C@_0DN@NCPDJLOG@?$CIthreadName?5?$DN?5jni_env?9?$DONewStrin@ 00000001800066d8     libsetenvstor001.obj
 0002:00001720       ??_C@_0FE@PFKODBGC@?$CIthreadObject?5?$DN?5jni_env?9?$DONewObj@ 0000000180006720     libsetenvstor001.obj
 0002:00001780       ??_C@_0ED@HOBAHHJI@?$CIthreadGlobalRef?5?$DN?5jni_env?9?$DONew@ 0000000180006780     libsetenvstor001.obj
 0002:000017d0       ??_C@_0FN@HNJJAHFC@jvmti_env?9?$DORunAgentThread?$CIagent@ 00000001800067d0     libsetenvstor001.obj
 0002:00001830       ??_C@_0EA@MOJDNKDF@Debuggee?5status?5sync?5aborted?5be@ 0000000180006830     libsetenvstor001.obj
 0002:00001870       ??_C@_0CO@PGPGMHBJ@No?5status?5sync?5occured?5for?5time@ 0000000180006870     libsetenvstor001.obj
 0002:000018a0       ??_C@_0CL@DOEBDPKJ@Debuggee?5was?5not?5suspended?5on?5s@ 00000001800068a0     libsetenvstor001.obj
 0002:000018d0       ??_C@_0EA@EEOEJAEN@status?5?$DN?5syncDebuggeeStatus?$CIjni@ 00000001800068d0     libsetenvstor001.obj
 0002:00001910       ??_C@_0BL@JBCFNBMB@nsk_jvmti_resetAgentData?$CI?$CJ@ 0000000180006910     libsetenvstor001.obj
 0002:00001930       ??_C@_0DN@NNGECJON@jvmti_env?9?$DOSetEventNotification@ 0000000180006930     libsetenvstor001.obj
 0002:00001970       ??_C@_0EL@LPBEELIP@s?2test?2hotspot?2jtreg?2vmTestbase@ 0000000180006970     libsetenvstor001.obj
 0002:000019c0       ??_C@_0CK@JDAMFDMJ@jvmti?9?$DOSetTag?$CIo?0?5tag?$CJ?5?$DN?$DN?5JVMTI_@ 00000001800069c0     libsetenvstor001.obj
 0002:000019f0       ??_C@_0CC@DAMNHKNI@Can?8t?5set?5tag?5?$CFli?5for?5object?5?$CFl@ 00000001800069f0     libsetenvstor001.obj
 0002:00001a18       ??_C@_0DL@HAJPNKEF@jvmti?9?$DOGetObjectHashCode?$CIo?0?5?$CGha@ 0000000180006a18     libsetenvstor001.obj
 0002:00001a58       ??_C@_0BL@JFPIEOBF@Can?8t?5get?5hash?5object?5?$CFlx?6@ 0000000180006a58     libsetenvstor001.obj
 0002:00001a78       ??_C@_0BG@DICPHBKN@setTag?3?5?$CF08x?5?$DM?9?5?$CF?53li@ 0000000180006a78     libsetenvstor001.obj
 0002:00001a90       ??_C@_0DH@FCEEBDMJ@?$CIs?5?$DN?5jni?9?$DOGetStringUTFChars?$CIsIn@ 0000000180006a90     libsetenvstor001.obj
 0002:00001ac8       ??_C@_0BJ@OKKGHDCN@Can?8t?5get?5string?5at?5?$CF?$CDp?6@ 0000000180006ac8     libsetenvstor001.obj
 0002:00001ae8       ??_C@_0BP@EKFLGGFJ@Can?8t?5get?5string?5at?5?$CF?$CDp?3?5null?6@ 0000000180006ae8     libsetenvstor001.obj
 0002:00001b08       ??_C@_06ICODBHCL@?5?1?1?5?$CFs@ 0000000180006b08     libsetenvstor001.obj
 0002:00001b10       ??_C@_0DB@KGFPLEGO@?$CIr?5?$DN?5jvmti?9?$DOGetTag?$CIo?0?5?$CGtag?$CJ?$CJ?5?$DN?$DN@ 0000000180006b10     libsetenvstor001.obj
 0002:00001b48       ??_C@_0CO@PDAGBCGJ@Can?8t?5GetTag?5for?5object?5?$CFlx?4?5Re@ 0000000180006b48     libsetenvstor001.obj
 0002:00001b78       ??_C@_0CH@HPEODOHC@TEST_BUG?3?5Max?4?5number?5of?5refs?5r@ 0000000180006b78     libsetenvstor001.obj
 0002:00001ba0       ??_C@_0DI@PHFCABIM@?$CIr?5?$DN?5jvmti?9?$DOGetTag?$CIfrom?0?5?$CGtagFr@ 0000000180006ba0     libsetenvstor001.obj
 0002:00001bd8       ??_C@_0DI@MDEGFNKD@TEST_BUG?3?5Can?8t?5GetTag?5for?5obje@ 0000000180006bd8     libsetenvstor001.obj
 0002:00001c10       ??_C@_0DE@MLELJAHM@?$CIr?5?$DN?5jvmti?9?$DOGetTag?$CIto?0?5?$CGtagTo?$CJ?$CJ@ 0000000180006c10     libsetenvstor001.obj
 0002:00001c48       ??_C@_0DD@INLPIDOF@Fill?5storage?5data?5with?5char?5?$CFc?5@ 0000000180006c48     libsetenvstor001.obj
 0002:00001c80       ??_C@_0GF@MOBJLGGA@s?2test?2hotspot?2jtreg?2vmTestbase@ 0000000180006c80     libsetenvstor001.obj
 0002:00001ce8       ??_C@_09IDOIEEAD@?5?5?4?4?4?5ok?6@ 0000000180006ce8     libsetenvstor001.obj
 0002:00001cf8       ??_C@_0CP@ENJMPPJC@Set?5local?5storage?5for?5current?5J@ 0000000180006cf8     libsetenvstor001.obj
 0002:00001d28       ??_C@_0CL@NPOOKEEL@jvmti?9?$DOSetEnvironmentLocalStora@ 0000000180006d28     libsetenvstor001.obj
 0002:00001d58       ??_C@_0CJ@CAAFGPKK@Get?5local?5storage?5for?5current?5J@ 0000000180006d58     libsetenvstor001.obj
 0002:00001d88       ??_C@_0DE@JDAMMKLE@jvmti?9?$DOGetEnvironmentLocalStora@ 0000000180006d88     libsetenvstor001.obj
 0002:00001dc0       ??_C@_0BJ@EBCAPHB@?5?5?4?4?4?5got?5storage?3?50x?$CFp?6@ 0000000180006dc0     libsetenvstor001.obj
 0002:00001de0       ??_C@_0GF@OGMDCHBA@Wrong?5storage?5pointer?5returned?5@ 0000000180006de0     libsetenvstor001.obj
 0002:00001e50       ??_C@_0GL@FDNIHHPN@Data?5changed?5in?5returned?5storag@ 0000000180006e50     libsetenvstor001.obj
 0002:00001ec0       ??_C@_0CC@HCPFMLEK@Wait?5for?5debugee?5to?5become?5read@ 0000000180006ec0     libsetenvstor001.obj
 0002:00001ee8       ??_C@_0DE@BIJKMJLC@?$DO?$DO?$DO?5Testcase?5?$CD3?3?5Check?5env?5stor@ 0000000180006ee8     libsetenvstor001.obj
 0002:00001f20       ??_C@_0N@POFOADDC@agent?5thread@ 0000000180006f20     libsetenvstor001.obj
 0002:00001f30       ??_C@_0BH@HPEOJMHL@Let?5debugee?5to?5finish?6@ 0000000180006f30     libsetenvstor001.obj
 0002:00001f48       ??_C@_0DI@OGIJFCJJ@?$DO?$DO?$DO?5Testcase?5?$CD2?3?5Check?5env?5stor@ 0000000180006f48     libsetenvstor001.obj
 0002:00001f80       ??_C@_0BB@ECBNOENI@VM_INIT?5callback@ 0000000180006f80     libsetenvstor001.obj
 0002:00001f98       ??_C@_0DJ@GKKAABOL@?$DO?$DO?$DO?5Testcase?5?$CD4?3?5Check?5env?5stor@ 0000000180006f98     libsetenvstor001.obj
 0002:00001fd8       ??_C@_0BC@BEKPBLPI@VM_DEATH?5callback@ 0000000180006fd8     libsetenvstor001.obj
 0002:00001ff0       ??_C@_0BL@OGOOPPCN@Disable?5events?3?5?$CFd?5events?6@ 0000000180006ff0     libsetenvstor001.obj
 0002:00002010       ??_C@_0BA@DDKAOGOI@?5?5?4?4?4?5disabled?6@ 0000000180007010     libsetenvstor001.obj
 0002:00002020       ??_C@_0CA@LDMJDFDO@Exit?5with?5FAIL?5exit?5status?3?5?$CFd?6@ 0000000180007020     libsetenvstor001.obj
 0002:00002040       ??_C@_0BC@PCOLJFHD@exit?$CISTATUS_FAIL?$CJ@ 0000000180007040     libsetenvstor001.obj
 0002:00002058       ??_C@_0CA@MNKGCBCG@nsk_jvmti_parseOptions?$CIoptions?$CJ@ 0000000180007058     libsetenvstor001.obj
 0002:00002078       ??_C@_0DN@MIAMNFPH@?$CIjvmti?5?$DN?5nsk_jvmti_createJVMTIE@ 0000000180007078     libsetenvstor001.obj
 0002:000020c0       ??_C@_0EC@ODFGFOAJ@jvmti?9?$DOSetEventCallbacks?$CI?$CGevent@ 00000001800070c0     libsetenvstor001.obj
 0002:00002108       ??_C@_0CL@PIACJIPK@nsk_jvmti_setAgentProc?$CIagentPro@ 0000000180007108     libsetenvstor001.obj
 0002:00002138       ??_C@_0CL@KPPJHIMN@?$DO?$DO?$DO?5Prepare?5storage?5data?5at?5poi@ 0000000180007138     libsetenvstor001.obj
 0002:00002168       ??_C@_0DC@BNDGKFCA@?$DO?$DO?$DO?5Testcase?5?$CD0?3?5Set?5env?5storag@ 0000000180007168     libsetenvstor001.obj
 0002:000021a0       ??_C@_0N@CNJBFCPG@JVM_OnLoad?$CI?$CJ@ 00000001800071a0     libsetenvstor001.obj
 0002:000021b0       ??_C@_0DE@EECAPNMP@?$DO?$DO?$DO?5Testcase?5?$CD1?3?5Check?5env?5stor@ 00000001800071b0     libsetenvstor001.obj
 0002:000021e8       ??_C@_0BK@EKNILGAD@Enable?5events?3?5?$CFd?5events?6@ 00000001800071e8     libsetenvstor001.obj
 0002:00002208       ??_C@_0P@BAMBNLJF@?5?5?4?4?4?5enabled?6@ 0000000180007208     libsetenvstor001.obj
 0002:00002230       ??_C@_1EC@JIJBPKFM@?$AAa?$AAp?$AAi?$AA?9?$AAm?$AAs?$AA?9?$AAw?$AAi?$AAn?$AA?9?$AAc?$AAo?$AAr?$AAe@ 0000000180007230     MSVCRT:thread_safe_statics.obj
 0002:00002278       ??_C@_1BK@MGMFAEKH@?$AAk?$AAe?$AAr?$AAn?$AAe?$AAl?$AA3?$AA2?$AA?4?$AAd?$AAl?$AAl@ 0000000180007278     MSVCRT:thread_safe_statics.obj
 0002:00002298       ??_C@_0BJ@JEBJOJFJ@SleepConditionVariableCS@ 0000000180007298     MSVCRT:thread_safe_statics.obj
 0002:000022b8       ??_C@_0BJ@PGPPEPCC@WakeAllConditionVariable@ 00000001800072b8     MSVCRT:thread_safe_statics.obj
 0002:000022d8       _pDefaultRawDllMain        00000001800072d8     MSVCRT:dll_dllmain.obj
 0002:000022d8       _pRawDllMain               00000001800072d8     MSVCRT:dll_dllmain.obj
 0002:000022e0       __xmm@ffffffffffffffffffffffffffffffff 00000001800072e0     MSVCRT:utility.obj
 0002:000022f0       _load_config_used          00000001800072f0     MSVCRT:loadcfg.obj
 0002:00002500       _tls_used                  0000000180007500     MSVCRT:tlssup.obj
 0002:00002528       __volatile_metadata        0000000180007528     <linker-defined>
 0002:00002930       __rtc_iaa                  0000000180007930     MSVCRT:initsect.obj
 0002:00002938       __rtc_izz                  0000000180007938     MSVCRT:initsect.obj
 0002:00002940       __rtc_taa                  0000000180007940     MSVCRT:initsect.obj
 0002:00002948       __rtc_tzz                  0000000180007948     MSVCRT:initsect.obj
 0002:00002950       _tls_start                 0000000180007950     MSVCRT:tlssup.obj
 0002:00002954       _Init_thread_epoch         0000000180007954     MSVCRT:thread_safe_statics.obj
 0002:00002958       _tls_end                   0000000180007958     MSVCRT:tlssup.obj
 0002:00003068       __IMPORT_DESCRIPTOR_KERNEL32 0000000180008068     kernel32:KERNEL32.dll
 0002:0000307c       __IMPORT_DESCRIPTOR_VCRUNTIME140 000000018000807c     vcruntime:VCRUNTIME140.dll
 0002:00003090       __IMPORT_DESCRIPTOR_api-ms-win-crt-heap-l1-1-0 0000000180008090     ucrt:api-ms-win-crt-heap-l1-1-0.dll
 0002:000030a4       __IMPORT_DESCRIPTOR_api-ms-win-crt-runtime-l1-1-0 00000001800080a4     ucrt:api-ms-win-crt-runtime-l1-1-0.dll
 0002:000030b8       __IMPORT_DESCRIPTOR_api-ms-win-crt-convert-l1-1-0 00000001800080b8     ucrt:api-ms-win-crt-convert-l1-1-0.dll
 0002:000030cc       __IMPORT_DESCRIPTOR_api-ms-win-crt-stdio-l1-1-0 00000001800080cc     ucrt:api-ms-win-crt-stdio-l1-1-0.dll
 0002:000030e0       __IMPORT_DESCRIPTOR_api-ms-win-crt-string-l1-1-0 00000001800080e0     ucrt:api-ms-win-crt-string-l1-1-0.dll
 0002:000030f4       __NULL_IMPORT_DESCRIPTOR   00000001800080f4     kernel32:KERNEL32.dll
 0003:00000040       _Init_global_epoch         0000000180009040     MSVCRT:thread_safe_statics.obj
 0003:00000050       __security_cookie          0000000180009050     MSVCRT:gs_cookie.obj
 0003:00000058       __security_cookie_complement 0000000180009058     MSVCRT:gs_cookie.obj
 0003:00000060       __scrt_native_dllmain_reason 0000000180009060     MSVCRT:utility.obj
 0003:00000068       __isa_available            0000000180009068     MSVCRT:cpu_disp.obj
 0003:0000006c       __isa_enabled              000000018000906c     MSVCRT:cpu_disp.obj
 0003:00000070       __memset_fast_string_threshold 0000000180009070     MSVCRT:cpu_disp.obj
 0003:00000078       __memset_nt_threshold      0000000180009078     MSVCRT:cpu_disp.obj
 0003:00000080       __scrt_ucrt_dll_is_in_use  0000000180009080     MSVCRT:ucrt_stubs.obj
 0003:00000090       g_wrongHeapCallbacks       0000000180009090     libsetenvstor001.obj
 0003:00000110       g_szTagInfo                0000000180009110     libsetenvstor001.obj
 0003:00002050       g_tagFlags                 000000018000b050     libsetenvstor001.obj
 0003:00002438       g_refsToVerifyCnt          000000018000b438     libsetenvstor001.obj
 0003:0000243c       g_fakeUserData             000000018000b43c     libsetenvstor001.obj
 0003:00002440       g_tagVisitCount            000000018000b440     libsetenvstor001.obj
 0003:000033e0       g_refsToVerify             000000018000c3e0     libsetenvstor001.obj
 0003:0001aae0       g_userDataError            0000000180023ae0     libsetenvstor001.obj
 0003:0001b088       ?_OptionsStorage@?1??__local_stdio_printf_options@@9@4_KA 0000000180024088     libsetenvstor001.obj
 0003:0001b648       _tls_index                 0000000180024648     MSVCRT:tlssup.obj
 0003:0001b650       __scrt_current_native_startup_state 0000000180024650     MSVCRT:utility.obj
 0003:0001b658       __scrt_native_startup_lock 0000000180024658     MSVCRT:utility.obj
 0003:0001b698       __scrt_debugger_hook_flag  0000000180024698     MSVCRT:utility_desktop.obj
 0003:0001b6a0       ?__type_info_root_node@@3U__type_info_node@@A 00000001800246a0     MSVCRT:tncleanup.obj
 0003:0001b6b0       ?_OptionsStorage@?1??__local_stdio_scanf_options@@9@4_KA 00000001800246b0     MSVCRT:default_local_stdio_options.obj
 0003:0001b6b8       __favor                    00000001800246b8     MSVCRT:cpu_disp.obj
 0003:0001b6c0       __dyn_tls_init_callback    00000001800246c0     <common>

 entry point at        0001:00002e70

 Static symbols

 0000:fffd9000       .debug$S                   0000000180000000     setenvstor001.exp
 0000:fffd9000       .debug$S                   0000000180000000     vcruntime:VCRUNTIME140.dll
 0000:fffd9000       .debug$S                   0000000180000000     vcruntime:VCRUNTIME140.dll
 0000:fffd9000       .debug$S                   0000000180000000     vcruntime:VCRUNTIME140.dll
 0000:fffd9000       .debug$S                   0000000180000000     vcruntime:VCRUNTIME140.dll
 0000:fffd9000       .debug$S                   0000000180000000     vcruntime:VCRUNTIME140.dll
 0000:fffd9000       .debug$S                   0000000180000000     vcruntime:VCRUNTIME140.dll
 0000:fffd9000       .debug$S                   0000000180000000     vcruntime:VCRUNTIME140.dll
 0000:fffd9000       .debug$S                   0000000180000000     ucrt:api-ms-win-crt-convert-l1-1-0.dll
 0000:fffd9000       .debug$S                   0000000180000000     ucrt:api-ms-win-crt-heap-l1-1-0.dll
 0000:fffd9000       .debug$S                   0000000180000000     ucrt:api-ms-win-crt-heap-l1-1-0.dll
 0000:fffd9000       .debug$S                   0000000180000000     ucrt:api-ms-win-crt-heap-l1-1-0.dll
 0000:fffd9000       .debug$S                   0000000180000000     ucrt:api-ms-win-crt-heap-l1-1-0.dll
 0000:fffd9000       .debug$S                   0000000180000000     ucrt:api-ms-win-crt-runtime-l1-1-0.dll
 0000:fffd9000       .debug$S                   0000000180000000     ucrt:api-ms-win-crt-runtime-l1-1-0.dll
 0000:fffd9000       .debug$S                   0000000180000000     ucrt:api-ms-win-crt-runtime-l1-1-0.dll
 0000:fffd9000       .debug$S                   0000000180000000     ucrt:api-ms-win-crt-runtime-l1-1-0.dll
 0000:fffd9000       .debug$S                   0000000180000000     ucrt:api-ms-win-crt-runtime-l1-1-0.dll
 0000:fffd9000       .debug$S                   0000000180000000     ucrt:api-ms-win-crt-runtime-l1-1-0.dll
 0000:fffd9000       .debug$S                   0000000180000000     ucrt:api-ms-win-crt-runtime-l1-1-0.dll
 0000:fffd9000       .debug$S                   0000000180000000     ucrt:api-ms-win-crt-runtime-l1-1-0.dll
 0000:fffd9000       .debug$S                   0000000180000000     ucrt:api-ms-win-crt-runtime-l1-1-0.dll
 0000:fffd9000       .debug$S                   0000000180000000     ucrt:api-ms-win-crt-runtime-l1-1-0.dll
 0000:fffd9000       .debug$S                   0000000180000000     ucrt:api-ms-win-crt-runtime-l1-1-0.dll
 0000:fffd9000       .debug$S                   0000000180000000     ucrt:api-ms-win-crt-runtime-l1-1-0.dll
 0000:fffd9000       .debug$S                   0000000180000000     ucrt:api-ms-win-crt-runtime-l1-1-0.dll
 0000:fffd9000       .debug$S                   0000000180000000     ucrt:api-ms-win-crt-runtime-l1-1-0.dll
 0000:fffd9000       .debug$S                   0000000180000000     ucrt:api-ms-win-crt-runtime-l1-1-0.dll
 0000:fffd9000       .debug$S                   0000000180000000     ucrt:api-ms-win-crt-runtime-l1-1-0.dll
 0000:fffd9000       .debug$S                   0000000180000000     ucrt:api-ms-win-crt-stdio-l1-1-0.dll
 0000:fffd9000       .debug$S                   0000000180000000     ucrt:api-ms-win-crt-stdio-l1-1-0.dll
 0000:fffd9000       .debug$S                   0000000180000000     ucrt:api-ms-win-crt-stdio-l1-1-0.dll
 0000:fffd9000       .debug$S                   0000000180000000     ucrt:api-ms-win-crt-stdio-l1-1-0.dll
 0000:fffd9000       .debug$S                   0000000180000000     ucrt:api-ms-win-crt-stdio-l1-1-0.dll
 0000:fffd9000       .debug$S                   0000000180000000     ucrt:api-ms-win-crt-stdio-l1-1-0.dll
 0000:fffd9000       .debug$S                   0000000180000000     ucrt:api-ms-win-crt-stdio-l1-1-0.dll
 0000:fffd9000       .debug$S                   0000000180000000     ucrt:api-ms-win-crt-stdio-l1-1-0.dll
 0000:fffd9000       .debug$S                   0000000180000000     ucrt:api-ms-win-crt-stdio-l1-1-0.dll
 0000:fffd9000       .debug$S                   0000000180000000     ucrt:api-ms-win-crt-stdio-l1-1-0.dll
 0000:fffd9000       .debug$S                   0000000180000000     ucrt:api-ms-win-crt-string-l1-1-0.dll
 0000:fffd9000       .debug$S                   0000000180000000     ucrt:api-ms-win-crt-string-l1-1-0.dll
 0000:fffd9000       .debug$S                   0000000180000000     ucrt:api-ms-win-crt-string-l1-1-0.dll
 0000:fffd9000       .debug$S                   0000000180000000     ucrt:api-ms-win-crt-string-l1-1-0.dll
 0000:fffd9000       .debug$S                   0000000180000000     ucrt:api-ms-win-crt-string-l1-1-0.dll
 0000:fffd9000       .debug$S                   0000000180000000     ucrt:api-ms-win-crt-string-l1-1-0.dll
 0000:fffd9000       .debug$S                   0000000180000000     ucrt:api-ms-win-crt-string-l1-1-0.dll
 0000:fffd9000       .debug$S                   0000000180000000     ucrt:api-ms-win-crt-string-l1-1-0.dll
 0000:fffd9000       .debug$S                   0000000180000000     kernel32:KERNEL32.dll
 0000:fffd9000       .debug$S                   0000000180000000     kernel32:KERNEL32.dll
 0000:fffd9000       .debug$S                   0000000180000000     kernel32:KERNEL32.dll
 0000:fffd9000       .debug$S                   0000000180000000     kernel32:KERNEL32.dll
 0000:fffd9000       .debug$S                   0000000180000000     kernel32:KERNEL32.dll
 0000:fffd9000       .debug$S                   0000000180000000     kernel32:KERNEL32.dll
 0000:fffd9000       .debug$S                   0000000180000000     kernel32:KERNEL32.dll
 0000:fffd9000       .debug$S                   0000000180000000     kernel32:KERNEL32.dll
 0000:fffd9000       .debug$S                   0000000180000000     kernel32:KERNEL32.dll
 0000:fffd9000       .debug$S                   0000000180000000     kernel32:KERNEL32.dll
 0000:fffd9000       .debug$S                   0000000180000000     kernel32:KERNEL32.dll
 0000:fffd9000       .debug$S                   0000000180000000     kernel32:KERNEL32.dll
 0000:fffd9000       .debug$S                   0000000180000000     kernel32:KERNEL32.dll
 0000:fffd9000       .debug$S                   0000000180000000     kernel32:KERNEL32.dll
 0000:fffd9000       .debug$S                   0000000180000000     kernel32:KERNEL32.dll
 0000:fffd9000       .debug$S                   0000000180000000     kernel32:KERNEL32.dll
 0000:fffd9000       .debug$S                   0000000180000000     kernel32:KERNEL32.dll
 0000:fffd9000       .debug$S                   0000000180000000     kernel32:KERNEL32.dll
 0000:fffd9000       .debug$S                   0000000180000000     kernel32:KERNEL32.dll
 0000:fffd9000       .debug$S                   0000000180000000     kernel32:KERNEL32.dll
 0000:fffd9000       .debug$S                   0000000180000000     kernel32:KERNEL32.dll
 0000:fffd9000       .debug$S                   0000000180000000     kernel32:KERNEL32.dll
 0000:fffd9000       .debug$S                   0000000180000000     kernel32:KERNEL32.dll
 0000:fffd9000       .debug$S                   0000000180000000     kernel32:KERNEL32.dll
 0000:fffd9000       .debug$S                   0000000180000000     kernel32:KERNEL32.dll
 0000:fffd9000       .debug$S                   0000000180000000     kernel32:KERNEL32.dll
 0000:fffd9000       .debug$S                   0000000180000000     kernel32:KERNEL32.dll
 0000:fffd9000       .debug$S                   0000000180000000     kernel32:KERNEL32.dll
 0001:00000f44       addRefToVerify             0000000180001f44 f   libsetenvstor001.obj
 0001:00000fb8       agentProc                  0000000180001fb8 f   libsetenvstor001.obj
 0001:00001048       agentThreadWrapper         0000000180002048 f   libsetenvstor001.obj
 0001:000012c4       checkEnvStorage            00000001800022c4 f   libsetenvstor001.obj
 0001:0000140c       check_option               000000018000240c f   libsetenvstor001.obj
 0001:00001654       file_basename              0000000180002654 f   libsetenvstor001.obj
 0001:000022ac       setEnvStorage              00000001800032ac f   libsetenvstor001.obj
 0001:0000237c       startAgentThreadWrapper    000000018000337c f   libsetenvstor001.obj
 0001:000026a8       syncDebuggeeStatus         00000001800036a8 f   libsetenvstor001.obj
 0001:00002930       capture_previous_context   0000000180003930 f   MSVCRT:gs_report.obj
 0001:000029a4       ?__scrt_initialize_thread_safe_statics@@YAHXZ 00000001800039a4 f   MSVCRT:thread_safe_statics.obj
 0001:00002a74       ?__scrt_uninitialize_thread_safe_statics@@YAXXZ 0000000180003a74 f   MSVCRT:thread_safe_statics.obj
 0001:00002b20       $$000000                   0000000180003b20     MSVCRT:amdsecgs.obj
 0001:00002b50       ?dllmain_crt_dispatch@@YAHQEAUHINSTANCE__@@KQEAX@Z 0000000180003b50 f   MSVCRT:dll_dllmain.obj
 0001:00002ba0       ?dllmain_crt_process_attach@@YAHQEAUHINSTANCE__@@QEAX@Z 0000000180003ba0 f   MSVCRT:dll_dllmain.obj
 0001:00002cb8       ?dllmain_crt_process_detach@@YAH_N@Z 0000000180003cb8 f   MSVCRT:dll_dllmain.obj
 0001:00002d3c       ?dllmain_dispatch@@YAHQEAUHINSTANCE__@@KQEAX@Z 0000000180003d3c f   MSVCRT:dll_dllmain.obj
 0001:00003750       $$000000                   0000000180004750     MSVCRT:guard_dispatch.obj
 0001:00003770       $$000000                   0000000180004770     MSVCRT:guard_xfg_dispatch.obj
 0001:00003786       ?fin$0@?0??dllmain_crt_process_attach@@YAHQEAUHINSTANCE__@@QEAX@Z@4HA 0000000180004786 f   MSVCRT:dll_dllmain.obj
 0001:0000379d       ?fin$0@?0??dllmain_crt_process_detach@@YAH_N@Z@4HA 000000018000479d f   MSVCRT:dll_dllmain.obj
 0001:000037b6       ?fin$1@?0??dllmain_crt_process_detach@@YAH_N@Z@4HA 00000001800047b6 f   MSVCRT:dll_dllmain.obj
 0001:000037ca       ?filt$0@?0??dllmain_dispatch@@YAHQEAUHINSTANCE__@@KQEAX@Z@4HA 00000001800047ca f   MSVCRT:dll_dllmain.obj
 0001:00003800       __scrt_is_nonwritable_in_current_image$filt$0 0000000180004800 f   MSVCRT:utility.obj
 0002:00000218       ?__scrt_initialize_tss_var@@3P6AHXZEA 0000000180005218     MSVCRT:thread_safe_statics.obj
 0002:00000340       ?opcLengths@@3QBEB         0000000180005340     libsetenvstor001.obj
 0002:00002218       GS_ExceptionPointers       0000000180007218     MSVCRT:gs_report.obj
 0002:00002960       $unwind$fprintf            0000000180007960     libsetenvstor001.obj
 0002:0000296c       $unwind$printf             000000018000796c     libsetenvstor001.obj
 0002:00002978       $unwind$?NewObject@JNIEnv_@@QEAAPEAV_jobject@@PEAV_jclass@@PEAU_jmethodID@@ZZ 0000000180007978     libsetenvstor001.obj
 0002:00002978       $unwind$nsk_lcomplain      0000000180007978     libsetenvstor001.obj
 0002:00002978       $unwind$nsk_ldisplay       0000000180007978     libsetenvstor001.obj
 0002:00002980       $unwind$nsk_lvdisplay      0000000180007980     libsetenvstor001.obj
 0002:00002980       $unwind$_RTC_Initialize    0000000180007980     MSVCRT:initsect.obj
 0002:00002980       $unwind$_RTC_Terminate     0000000180007980     MSVCRT:initsect.obj
 0002:00002980       $unwind$?__scrt_initialize_thread_safe_statics@@YAHXZ 0000000180007980     MSVCRT:thread_safe_statics.obj
 0002:0000298c       $unwind$nsk_complain       000000018000798c     libsetenvstor001.obj
 0002:0000298c       $unwind$nsk_printf         000000018000798c     libsetenvstor001.obj
 0002:00002994       $unwind$nsk_lvcomplain     0000000180007994     libsetenvstor001.obj
 0002:000029ac       $unwind$nsk_ltrace         00000001800079ac     libsetenvstor001.obj
 0002:000029ac       $unwind$__report_gsfailure 00000001800079ac     MSVCRT:gs_report.obj
 0002:000029b4       $unwind$agentProc          00000001800079b4     libsetenvstor001.obj
 0002:000029b4       $unwind$callbackVMInit     00000001800079b4     libsetenvstor001.obj
 0002:000029b4       $unwind$nsk_lvtrace        00000001800079b4     libsetenvstor001.obj
 0002:000029b4       $unwind$__raise_securityfailure 00000001800079b4     MSVCRT:gs_report.obj
 0002:000029b4       $unwind$__scrt_initialize_crt 00000001800079b4     MSVCRT:utility.obj
 0002:000029b4       $unwind$__scrt_initialize_onexit_tables 00000001800079b4     MSVCRT:utility.obj
 0002:000029b4       $unwind$__scrt_release_startup_lock 00000001800079b4     MSVCRT:utility.obj
 0002:000029b4       $unwind$__scrt_uninitialize_crt 00000001800079b4     MSVCRT:utility.obj
 0002:000029b4       $unwind$_onexit            00000001800079b4     MSVCRT:utility.obj
 0002:000029bc       $unwind$nsk_lverify        00000001800079bc     libsetenvstor001.obj
 0002:000029cc       $unwind$nsk_vprintf        00000001800079cc     libsetenvstor001.obj
 0002:000029dc       $unwind$?nsk_jni_lverify@@YAHHPEAUJNIEnv_@@HQEBDH1ZZ 00000001800079dc     libsetenvstor001.obj
 0002:000029f0       $unwind$?nsk_jni_check_exception@@YAHPEAUJNIEnv_@@QEBDH@Z 00000001800079f0     libsetenvstor001.obj
 0002:00002a0c       $unwind$nsk_jvmti_parseOptions 0000000180007a0c     libsetenvstor001.obj
 0002:00002a28       $unwind$nsk_jvmti_createJVMTIEnv 0000000180007a28     libsetenvstor001.obj
 0002:00002a3c       $unwind$check_option       0000000180007a3c     libsetenvstor001.obj
 0002:00002a3c       $unwind$nsk_jvmti_waitForSync 0000000180007a3c     libsetenvstor001.obj
 0002:00002a3c       $unwind$_DllMainCRTStartup 0000000180007a3c     MSVCRT:dll_dllmain.obj
 0002:00002a4c       $unwind$Java_nsk_jvmti_unit_FollowReferences_FollowRefObjects_resetTags 0000000180007a4c     libsetenvstor001.obj
 0002:00002a4c       $unwind$addRefToVerify     0000000180007a4c     libsetenvstor001.obj
 0002:00002a4c       $unwind$nsk_jvmti_resetAgentData 0000000180007a4c     libsetenvstor001.obj
 0002:00002a4c       $unwind$nsk_jvmti_resumeSync 0000000180007a4c     libsetenvstor001.obj
 0002:00002a4c       $unwind$__scrt_initialize_default_local_stdio_options 0000000180007a4c     MSVCRT:default_local_stdio_options.obj
 0002:00002a4c       $unwind$?dllmain_crt_dispatch@@YAHQEAUHINSTANCE__@@KQEAX@Z 0000000180007a4c     MSVCRT:dll_dllmain.obj
 0002:00002a4c       $unwind$DllMain            0000000180007a4c     MSVCRT:dll_dllmain_stub.obj
 0002:00002a4c       $unwind$__GSHandlerCheck   0000000180007a4c     MSVCRT:gshandler.obj
 0002:00002a4c       $unwind$?__scrt_uninitialize_thread_safe_statics@@YAXXZ 0000000180007a4c     MSVCRT:thread_safe_statics.obj
 0002:00002a4c       $unwind$__scrt_acquire_startup_lock 0000000180007a4c     MSVCRT:utility.obj
 0002:00002a4c       $unwind$__scrt_dllmain_after_initialize_c 0000000180007a4c     MSVCRT:utility.obj
 0002:00002a4c       $unwind$__scrt_dllmain_before_initialize_c 0000000180007a4c     MSVCRT:utility.obj
 0002:00002a4c       $unwind$__scrt_dllmain_crt_thread_attach 0000000180007a4c     MSVCRT:utility.obj
 0002:00002a4c       $unwind$__scrt_dllmain_crt_thread_detach 0000000180007a4c     MSVCRT:utility.obj
 0002:00002a4c       $unwind$__scrt_dllmain_uninitialize_c 0000000180007a4c     MSVCRT:utility.obj
 0002:00002a4c       $unwind$__scrt_dllmain_uninitialize_critical 0000000180007a4c     MSVCRT:utility.obj
 0002:00002a4c       $unwind$atexit             0000000180007a4c     MSVCRT:utility.obj
 0002:00002a54       $unwind$nsk_jvmti_enableEvents 0000000180007a54     libsetenvstor001.obj
 0002:00002a6c       $unwind$nsk_jvmti_lverify  0000000180007a6c     libsetenvstor001.obj
 0002:00002a80       $unwind$exitOnError        0000000180007a80     libsetenvstor001.obj
 0002:00002a90       $unwind$Java_nsk_share_jvmti_ArgumentHandler_getAgentOptionsString 0000000180007a90     libsetenvstor001.obj
 0002:00002aa4       $unwind$Java_nsk_jvmti_unit_FollowReferences_FollowRefObjects_getTag 0000000180007aa4     libsetenvstor001.obj
 0002:00002aa4       $unwind$Java_nsk_share_jvmti_DebugeeClass_checkStatus 0000000180007aa4     libsetenvstor001.obj
 0002:00002aa4       $unwind$agentThreadWrapper 0000000180007aa4     libsetenvstor001.obj
 0002:00002ab4       $unwind$startAgentThreadWrapper 0000000180007ab4     libsetenvstor001.obj
 0002:00002ad0       $unwind$syncDebuggeeStatus 0000000180007ad0     libsetenvstor001.obj
 0002:00002ad0       $unwind$__scrt_dllmain_exception_filter 0000000180007ad0     MSVCRT:utility.obj
 0002:00002ae4       $unwind$Java_nsk_share_jvmti_DebugeeClass_resetAgentData 0000000180007ae4     libsetenvstor001.obj
 0002:00002aec       $unwind$MA_checkStatus     0000000180007aec     libsetenvstor001.obj
 0002:00002b00       $unwind$Java_nsk_jvmti_unit_FollowReferences_FollowRefObjects_setTag 0000000180007b00     libsetenvstor001.obj
 0002:00002b18       $unwind$Java_nsk_jvmti_unit_FollowReferences_FollowRefObjects_addRefToVerify 0000000180007b18     libsetenvstor001.obj
 0002:00002b34       $unwind$Agent_Initialize   0000000180007b34     libsetenvstor001.obj
 0002:00002b54       $unwind$setEnvStorage      0000000180007b54     libsetenvstor001.obj
 0002:00002b68       $unwind$checkEnvStorage    0000000180007b68     libsetenvstor001.obj
 0002:00002b80       $unwind$callbackVMDeath    0000000180007b80     libsetenvstor001.obj
 0002:00002b8c       $unwind$capture_previous_context 0000000180007b8c     MSVCRT:gs_report.obj
 0002:00002b98       $unwind$__GSHandlerCheckCommon 0000000180007b98     MSVCRT:gshandler.obj
 0002:00002ba0       $xdatasym                  0000000180007ba0     MSVCRT:amdsecgs.obj
 0002:00002ba4       $unwind$?dllmain_crt_process_attach@@YAHQEAUHINSTANCE__@@QEAX@Z 0000000180007ba4     MSVCRT:dll_dllmain.obj
 0002:00002be0       $unwind$?fin$0@?0??dllmain_crt_process_attach@@YAHQEAUHINSTANCE__@@QEAX@Z@4HA 0000000180007be0     MSVCRT:dll_dllmain.obj
 0002:00002be0       $unwind$?fin$0@?0??dllmain_crt_process_detach@@YAH_N@Z@4HA 0000000180007be0     MSVCRT:dll_dllmain.obj
 0002:00002be0       $unwind$?fin$1@?0??dllmain_crt_process_detach@@YAH_N@Z@4HA 0000000180007be0     MSVCRT:dll_dllmain.obj
 0002:00002be8       $unwind$?dllmain_crt_process_detach@@YAH_N@Z 0000000180007be8     MSVCRT:dll_dllmain.obj
 0002:00002c3c       $unwind$?dllmain_dispatch@@YAHQEAUHINSTANCE__@@KQEAX@Z 0000000180007c3c     MSVCRT:dll_dllmain.obj
 0002:00002c64       $unwind$?filt$0@?0??dllmain_dispatch@@YAHQEAUHINSTANCE__@@KQEAX@Z@4HA 0000000180007c64     MSVCRT:dll_dllmain.obj
 0002:00002c6c       $unwind$__scrt_is_nonwritable_in_current_image 0000000180007c6c     MSVCRT:utility.obj
 0002:00002c8c       $unwind$__scrt_is_nonwritable_in_current_image$filt$0 0000000180007c8c     MSVCRT:utility.obj
 0002:00002c94       $unwind$__scrt_fastfail    0000000180007c94     MSVCRT:utility_desktop.obj
 0002:00002ca4       $unwind$__security_init_cookie 0000000180007ca4     MSVCRT:gs_support.obj
 0002:00002cb0       $unwind$__isa_available_init 0000000180007cb0     MSVCRT:cpu_disp.obj
 0002:00002cc0       $xdatasym                  0000000180007cc0     MSVCRT:guard_dispatch.obj
 0002:00002cc8       $xdatasym                  0000000180007cc8     MSVCRT:guard_xfg_dispatch.obj
 0002:00002cd0       .edata                     0000000180007cd0     setenvstor001.exp
 0002:00002cf8       rgpv                       0000000180007cf8     setenvstor001.exp
 0002:00002d38       rgszName                   0000000180007d38     setenvstor001.exp
 0002:00002d78       rgwOrd                     0000000180007d78     setenvstor001.exp
 0002:00002d98       szName                     0000000180007d98     setenvstor001.exp
 0002:00002daa       $N00001                    0000000180007daa     setenvstor001.exp
 0002:00002db9       $N00002                    0000000180007db9     setenvstor001.exp
 0002:00002dc6       $N00003                    0000000180007dc6     setenvstor001.exp
 0002:00002e0b       $N00004                    0000000180007e0b     setenvstor001.exp
 0002:00002e48       $N00005                    0000000180007e48     setenvstor001.exp
 0002:00002e90       $N00006                    0000000180007e90     setenvstor001.exp
 0002:00002ed0       $N00007                    0000000180007ed0     setenvstor001.exp
 0002:00002f0d       $N00008                    0000000180007f0d     setenvstor001.exp
 0002:00002f48       $N00009                    0000000180007f48     setenvstor001.exp
 0002:00002f76       $N00010                    0000000180007f76     setenvstor001.exp
 0002:00002fa7       $N00011                    0000000180007fa7     setenvstor001.exp
 0002:00002fd6       $N00012                    0000000180007fd6     setenvstor001.exp
 0002:00003005       $N00013                    0000000180008005     setenvstor001.exp
 0002:0000303a       $N00014                    000000018000803a     setenvstor001.exp
 0002:00003049       $N00015                    0000000180008049     setenvstor001.exp
 0002:00003059       $N00016                    0000000180008059     setenvstor001.exp
 0002:000034ba       .idata$6                   00000001800084ba     kernel32:KERNEL32.dll
 0002:0000351e       .idata$6                   000000018000851e     vcruntime:VCRUNTIME140.dll
 0002:000036b0       .idata$6                   00000001800086b0     ucrt:api-ms-win-crt-heap-l1-1-0.dll
 0002:000036d0       .idata$6                   00000001800086d0     ucrt:api-ms-win-crt-runtime-l1-1-0.dll
 0002:000036f2       .idata$6                   00000001800086f2     ucrt:api-ms-win-crt-convert-l1-1-0.dll
 0002:00003714       .idata$6                   0000000180008714     ucrt:api-ms-win-crt-stdio-l1-1-0.dll
 0002:00003734       .idata$6                   0000000180008734     ucrt:api-ms-win-crt-string-l1-1-0.dll
 0003:00000000       ?codeAttributeName@@3PEBDEB 0000000180009000     libsetenvstor001.obj
 0003:00000008       ?lineNumberAttributeName@@3PEBDEB 0000000180009008     libsetenvstor001.obj
 0003:00000010       ?localVarAttributeName@@3PEBDEB 0000000180009010     libsetenvstor001.obj
 0003:00000018       ?localVarTypeAttributeName@@3PEBDEB 0000000180009018     libsetenvstor001.obj
 0003:00000020       ?stackMapAttributeName@@3PEBDEB 0000000180009020     libsetenvstor001.obj
 0003:00000028       ?callBytes@@3PAEA          0000000180009028     libsetenvstor001.obj
 0003:0000002c       ?allocBytes@@3PAEA         000000018000902c     libsetenvstor001.obj
 0003:00000030       events                     0000000180009030     libsetenvstor001.obj
 0003:00000038       initialStorage             0000000180009038     libsetenvstor001.obj
 0003:0001aaf0       storageData                0000000180023af0     libsetenvstor001.obj
 0003:0001aef0       nsk_context                0000000180023ef0     libsetenvstor001.obj
 0003:0001aefc       redefineAttempted          0000000180023efc     libsetenvstor001.obj
 0003:0001af00       redefineSucceed            0000000180023f00     libsetenvstor001.obj
 0003:0001af04       agentFailed                0000000180023f04     libsetenvstor001.obj
 0003:0001af08       agentThread                0000000180023f08     libsetenvstor001.obj
 0003:0001af10       context                    0000000180023f10     libsetenvstor001.obj
 0003:0001afc8       agentThreadProc            0000000180023fc8     libsetenvstor001.obj
 0003:0001afd0       agentThreadArg             0000000180023fd0     libsetenvstor001.obj
 0003:0001afd8       agent_data                 0000000180023fd8     libsetenvstor001.obj
 0003:0001afe8       jvmti_env                  0000000180023fe8     libsetenvstor001.obj
 0003:0001aff0       jvm                        0000000180023ff0     libsetenvstor001.obj
 0003:0001aff8       jni_env                    0000000180023ff8     libsetenvstor001.obj
 0003:0001b000       currentAgentStatus         0000000180024000     libsetenvstor001.obj
 0003:0001b004       ?codeAttributeIndex@@3GA   0000000180024004     libsetenvstor001.obj
 0003:0001b008       checkStatus_func           0000000180024008     libsetenvstor001.obj
 0003:0001b010       ?lineNumberAttributeIndex@@3GA 0000000180024010     libsetenvstor001.obj
 0003:0001b014       ?localVarAttributeIndex@@3GA 0000000180024014     libsetenvstor001.obj
 0003:0001b018       ?localVarTypeAttributeIndex@@3GA 0000000180024018     libsetenvstor001.obj
 0003:0001b01c       ?stackMapAttributeIndex@@3GA 000000018002401c     libsetenvstor001.obj
 0003:0001b020       ?stackFrameOffset@@3GA     0000000180024020     libsetenvstor001.obj
 0003:0001b024       ?mode@@3HA                 0000000180024024     libsetenvstor001.obj
 0003:0001b028       ?orig@@3PEBEEB             0000000180024028     libsetenvstor001.obj
 0003:0001b030       ?gen@@3PEAEEA              0000000180024030     libsetenvstor001.obj
 0003:0001b038       ?inputPos@@3PEAEEA         0000000180024038     libsetenvstor001.obj
 0003:0001b040       ?endPos@@3PEBEEB           0000000180024040     libsetenvstor001.obj
 0003:0001b048       ?genPos@@3PEAEEA           0000000180024048     libsetenvstor001.obj
 0003:0001b050       ?markPos@@3PEAEEA          0000000180024050     libsetenvstor001.obj
 0003:0001b058       ?constantPool@@3PEAPEADEA  0000000180024058     libsetenvstor001.obj
 0003:0001b060       ?constantPoolSize@@3GA     0000000180024060     libsetenvstor001.obj
 0003:0001b064       ?constantPoolCount@@3GA    0000000180024064     libsetenvstor001.obj
 0003:0001b068       ?zeroBytes@@3PAEA          0000000180024068     libsetenvstor001.obj
 0003:0001b06c       ?codeLength@@3IA           000000018002406c     libsetenvstor001.obj
 0003:0001b070       ?map@@3PEAIEA              0000000180024070     libsetenvstor001.obj
 0003:0001b078       ?widening@@3PEACEA         0000000180024078     libsetenvstor001.obj
 0003:0001b080       timeout                    0000000180024080     libsetenvstor001.obj
 0003:0001b090       GS_ExceptionRecord         0000000180024090     MSVCRT:gs_report.obj
 0003:0001b130       GS_ContextRecord           0000000180024130     MSVCRT:gs_report.obj
 0003:0001b600       ?g_tss_cv@@3U_RTL_CONDITION_VARIABLE@@A 0000000180024600     MSVCRT:thread_safe_statics.obj
 0003:0001b608       ?g_tss_event@@3PEAXEA      0000000180024608     MSVCRT:thread_safe_statics.obj
 0003:0001b610       ?g_tss_mutex@@3U_RTL_CRITICAL_SECTION@@A 0000000180024610     MSVCRT:thread_safe_statics.obj
 0003:0001b638       ?g_sleep_condition_variable_cs@@3P6AHPEAU_RTL_CONDITION_VARIABLE@@PEAU_RTL_CRITICAL_SECTION@@K@ZEA 0000000180024638     MSVCRT:thread_safe_statics.obj
 0003:0001b640       ?g_wake_all_condition_variable@@3P6AXPEAU_RTL_CONDITION_VARIABLE@@@ZEA 0000000180024640     MSVCRT:thread_safe_statics.obj
 0003:0001b64c       ?__proc_attached@@3HA      000000018002464c     MSVCRT:dll_dllmain.obj
 0003:0001b660       ?is_initialized_as_dll@@3_NA 0000000180024660     MSVCRT:utility.obj
 0003:0001b661       ?module_local_atexit_table_initialized@@3_NA 0000000180024661     MSVCRT:utility.obj
 0003:0001b668       ?module_local_atexit_table@@3U_onexit_table_t@@A 0000000180024668     MSVCRT:utility.obj
 0003:0001b680       ?module_local_at_quick_exit_table@@3U_onexit_table_t@@A 0000000180024680     MSVCRT:utility.obj
